:1000000000308A009F280000243084000008031973
:1000100016280230F800F701F70B0C28F80B0B2814
:100020009730F700F70B1228800B0928003483164D
:100030008511831285156430A40004208316851170
:10004000831285116430A40004200034A208031D2B
:1000500042288316051283120516FA30A4000420E4
:1000600083160512831205120330A300FA30A40090
:100070000420A30B36288316051283120516FA30C6
:10008000A4000420A20803195C2883160512831219
:100090000516FA30A40004208316051283120512F7
:1000A000FA30A40004208316051283120516FA30D4
:1000B000A4000420A2034228F228A60803197C28E1
:1000C000831605118312051100000000A51B6A2884
:1000D00085106B288514831685100000000005111B
:1000E0008312051500000000831605118312051107
:1000F0000310A50DA6035D28003483160510831296
:10010000051400000000831605108312051000007E
:1001100000002208A5000830A6005D202308A500E5
:100120000830A6005D202408A5000830A6005D2048
:1001300000000000831605108312051400348401AA
:100140001F30830583161F149F141F159F117030D5
:100150008F0006118312061583160108C739083867
:100160008100831290010030F80092000030831665
:10017000920083121F108316861183128611172096
:100180008316061600308312061A0130F700770D29
:10019000A300A30DA30DF830A30583168616003027
:1001A0008312861A0130F700F70DF70DFC30F705C2
:1001B00077082307A5008316051700308312051B57
:1001C0000130F7000310F70D77082507A700831605
:1001D000851700308312851B01302707A1000430EA
:1001E000A2002628A201A3019630A4007D20A2012E
:1001F000A3010430A4007D20A2010C30A300113023
:10020000A4007D20A201A3019230A4007D2017202C
:100210001720831606148312061C172983168611CD
:100220008312861183160512831205161F29831661
:10023000861183128615831605128312051208296A
:02024000630059
:02400E00703F01
:00000001FF
